:0300000002000EED
:03000300020028D0
:20000B0002001F75810AD2AFD2A912002B80FE12001B80FB758CDC758A00050832050832FB
:20002B007400F50A7400F509748075F025C0E0C0F01200AA15811581E5081200F87B001296
:20004B0000EF12014545F0700302005A0200437400F50812006812008C02004322E5090423
:20006B00F50914E50975F0007B327C0012017145F0700302008B7400F509E50A4401F50A89
:20008B0022E50A540175F0007B007C0012014E45F070030200A9B297E50A54FEF50A2278BC
:2000AB00FB1200CD8603088604748075F07012010112013B758921F58DF58B758859759891
:2000CB005222C82581C822C92581C97A0022D083D082CF2581F581CFC082C08322CF2581FA
:2000EB00F581CF227C00CB30E7011CCB2275F00030E70215F022C002C001AAF0F97E007D70
:20010B00007F11C3E933F9EA33FADF08F5F0E9D001D00222ED33FDEE33FEC3ED9BF5F0EE81
:20012B009C40E0ADF0FED380DB14B4FF0215F022120134F4C5F0F4C5F0221201786009E4AC
:20014B00F5F02212017860F7E4F5F0042212017840F680EB12017840EF70E480EB1201788C
:20016B0040DD70E480D912017850DD80D2C5F0C39C7003E5F09B22FBE493CB22FCE493FBBA
:0E018B00740193CC22FAE493F9740193CA2212
:00000001FF
